:10000000A0011D299000250884002308A520841341
:100010000005181C2306031920281008031D1828A2
:100020001608FF3E031C21280A30BE20160821288E
:10003000100AFF3003192028100B20281708212848
:100040009909031019180314182991019000A11798
:1000500027308F001030382003308F00E8303820F0
:100060008F01643038208F010A303820100843286F
:100070008E0011088D0010088C00E0200C08031D74
:10008000A113A11B0800303EA0186F289300861111
:100090008316861183123A308D009830CC2086105A
:1000A0008316861083123330920083160F30860534
:1000B000831283200F308D00DC30CC2083203C3035
:1000C000CB20832022309200832020306E200C3001
:1000D0006E2006306E20A01413086F2820149200A2
:1000E000201C7D288610033C031C822882203E3081
:1000F0008D008030CC20031408002014FE3C03192E
:1001000018298614201C20100F3086051208F0399B
:1001100086048615920E8611201883282830CB205D
:1001200003140800A300A8200C080D0403191829C3
:10013000122184132308800664009E289F288C0ABD
:1001400003198D0F9C28800618298417800418290C
:10015000FF3A841780051829890083160814831232
:100160000808182988008316081555308900AA3018
:10017000890088148818BA28081118298F018E0060
:10018000FF308E07031C8F07031C182903308D00D6
:10019000DF30CC20C0288D01E83E8C008D09FC307A
:1001A000031CD5288C070318D2288C0764008D0FF8
:1001B000D2280C18DB288C1CDF280000DF28080060
:1001C00010309200910190010D0D900D910D0E08CF
:1001D00090020F08031C0F0F91020318F6280E0857
:1001E00090070F0803180F0F910703108C0D8D0D4A
:1001F000920BE4280C081829103094008D018C0112
:10020000930C920C031C0A290E088C070F08031884
:100210000F0F8D078D0C8C0C910C900C940B0029FA
:10022000100818298C098D098C0A03198D0A0800F9
:1002300083130313831264000800831605148514C6
:1002400005168312A830B5000130B6000030AC208E
:10025000BD000130AC20B300B401F430B30701306D
:100260000318013EB4070230AC20BC000330AC20C0
:10027000B100B201F430B10701300318013EB207FA
:1002800086108316861083120610831606108312BA
:1002900006118316061183128511831685118312A8
:1002A00006118316061183120430C5004130B900CF
:1002B000BA01C830BE20FE30442001304420453011
:1002C00044205230442032304420303044203030FA
:1002D00044203130442020304420503044206130CC
:1002E0004420633044206B3044202030442032309E
:1002F00044202E3044203230442003308F00E83038
:10030000BF20AC225C2A0530A5001030A300980164
:10031000FF30960097010130990042080220C20088
:100320000318D4290530A5000130A30098010A3034
:10033000960002309700013099003E080220BE006E
:1003400003181A2A0530A5000230A30098010A30CC
:10035000960002309700013099003F080220BF004C
:100360000318292A0530A5000430A3009801FF30A6
:10037000960097010130990040080220C000031840
:10038000832A0530A5000430A30001309800FF3017
:10039000960097010130990041080220C10003181E
:1003A0005C2A6430BE2083290430C5076400053010
:1003B00045020318DC29DE29C501DE296400450851
:1003C000043C0319E7294130B900BA01EA29423057
:1003D000B900BA01003045079E009F019F0D1E081D
:1003E000AC20BD00013045079E009F019F0D1E08F7
:1003F000AC20B300B401F430B30701300318013E60
:10040000B407023045079E009F019F0D1E08AC20D7
:10041000BC00033045079E009F019F0D1E08AC20C5
:10042000B100B201F430B10701300318013EB20748
:10043000AC225C2A64003D083F3C0319382ABD0AFF
:1004400064003C083F3C03193F2ABC0AAC22FB2253
:100450005C2A64003D08003C0319462ABD03640081
:100460003C08003C0319512ABC03AC22FB225C2A45
:10047000B30A0319B40ABD01AC220E23202AB10A23
:100480000319B20ABC01AC220E23262A0130B302A2
:100490000030031C013EB4023F30BD00AC220E23ED
:1004A0002F2A0130B1020030031C013EB2023F305E
:1004B000BC00AC220E23352A22145230B700B801FA
:1004C0003D08BB0002303307AD0034080318013E7D
:1004D000AE00061483160610831239230610831605
:1004E000061083123C08BB003108AD003208AE0094
:1004F000851583168511831239238511831685117D
:100500008312DE22832922105430B700B8013C0840
:10051000BB0002303107AD0032080318013EAE00C7
:10052000851583168511831239238511831685114C
:1005300083123D08BB003308AD003408AE0006143A
:1005400083160610831239230610831606108312B1
:10055000DE2283296300AA2AF4303302AF0001307F
:10056000031C013E3402B00020309200033093009F
:100570002F088E0030088F00FC20A7001108A8006B
:100580007D30920093013D088E008F01FC20A90070
:100590001108AA0029088C002A088D000A308E0054
:1005A0008F01E0209E000D089F0027081E07AB006A
:1005B00028080318013E1F07AC000800FE30442045
:1005C0000130442037084420583044202030442053
:1005D000043025202C0891002B08262020304420B0
:1005E0006B304420483044207A304420203044206E
:1005F000390844200800003045079E009F019F0DE8
:100600001E0889003D08B220023045079E009F0168
:100610009F0D1E0889003C08B220080000304507E5
:100620009E009F019F0D1E0889003D08B220F430F6
:100630003302C400013045079E009F019F0D1E0834
:1006400089004408B220023045079E009F019F0D9B
:100650001E0889003C08B220F4303102C300033088
:1006600045079E009F019F0D1E0889004308B22088
:1006700008003B1B06153B1F0611C623BB1A0615B7
:10068000BB1E0611C6233B1A06153B1E0611C623C8
:10069000BB190615BB1D0611C6233B1906153B1DCC
:1006A0000611C623BB180615BB1C0611C6233B1832
:1006B00006153B1C0611C623AE180615AE1C061106
:1006C000C6232E1806152E1C0611C623AD1B0615B3
:1006D000AD1F0611C6232D1B06152D1F0611C6239F
:1006E000AD1A0615AD1E0611C6232D1A06152D1EB0
:1006F0000611C623AD190615AD1D0611C6232D1909
:1007000006152D1D0611C623AD180615AD1C0611C4
:10071000C6232D1806152D1C0611C62336190615DD
:10072000361D0611C623B6180615B61C0611C623BB
:1007300036180615361C0611C623B51B0615B51F3F
:100740000611C623351B0615351F0611C623B51A1B
:100750000615B51E0611C623351A0615351E0611D7
:10076000C623B5190615B51D0611C623351906157C
:10077000351D0611C623B5180615B51C0611C6236E
:1007800035180615351C0611C623080005308C00E7
:0C0790008D010630840002309220080029
:02400E00F53F7C
:1042000008002A0018000F0008002A0018000F00FC
:00000001FF
